:020000040800F2
:1000000080330020CD010008CD29000831230008ED
:10001000C92900084D040008E13300080000000071
:10002000000000000000000000000000F52D0008A6
:100030001D05000800000000D1290008C92E000895
:10004000E7010008E7010008E7010008E7010008F0
:10005000E7010008E7010008E7010008E7010008E0
:10006000E7010008E7010008E7010008E7010008D0
:10007000E7010008E7010008E7010008E7010008C0
:100080000D050008E7010008E7010008E701000886
:10009000E7010008E7010008E7010008E7010008A0
:1000A000E7010008E7010008E7010008E701000890
:1000B000D52E0008E7010008E7010008E701000865
:1000C000E7010008E7010008E7010008E701000870
:1000D000E7010008C1330008D1330008E701000838
:1000E000E7010008E7010008E7010008E701000850
:1000F000E7010008E7010008E7010008E701000840
:10010000E7010008E7010008E7010008E70100082F
:10011000E7010008E7010008E7010008E70100081F
:10012000E7010008E7010008E7010008E70100080F
:1001300000F002F800F03AF80AA090E8000C8244BF
:100140008344AAF10107DA4501D100F02FF8AFF29C
:10015000090EBAE80F0013F0010F18BFFB1A43F0A5
:1001600001031847D43C0000F43C0000103A24BFBF
:1001700078C878C1FAD8520724BF30C830C144BF0C
:1001800004680C607047000000230024002500264E
:10019000103A28BF78C1FBD8520728BF30C148BFEA
:1001A0000B6070471FB51FBD10B510BD00F0E8F81B
:1001B0001146FFF7F7FF03F0DFFB00F006F903B489
:1001C000FFF7F2FF03BC03F0B5F9000009488047D0
:1001D00009480047FEE7FEE7FEE7FEE7FEE7FEE729
:1001E000FEE7FEE7FEE7FEE704480549054A064B41
:1001F00070470000D12E000831010008802D00203A
:1002000080330020802F0020802F00207047B2F123
:1002100020030AD5C2F1200320FA02F001FA03F309
:1002200021FA02F140EA0300704721FA03F04FF08F
:1002300000017047032A40F2308010F0030C00F0F8
:10024000158011F8013BBCF1020F624498BF11F810
:1002500001CB00F8013B38BF11F8013BA2F10402C9
:1002600098BF00F801CB38BF00F8013B11F0030341
:1002700000F02580083AC0F0088051F8043B083AA5
:1002800051F804CBA0E80810F5E7121D5CBF51F847
:10029000043B40F8043BAFF30080D20724BF11F8C1
:1002A000013B11F801CB48BF11F8012B24BF00F826
:1002B000013B00F801CB48BF00F8012B704710B597
:1002C000203AC0F00B80B1E81850203AA0E818504E
:1002D000B1E81850A0E81850BFF4F5AF5FEA027C0F
:1002E00024BFB1E81850A0E8185044BF18C918C07E
:1002F000BDE810405FEA827C24BF51F8043B40F81F
:10030000043B08BF7047D20728BF31F8023B48BF03
:1003100011F8012B28BF20F8023B48BF00F8012B41
:1003200070474FF0000200B51346944696462039B8
:1003300022BFA0E80C50A0E80C50B1F12001BFF49E
:10034000F7AF090728BFA0E80C5048BF0CC05DF804
:1003500004EB890028BF40F8042B08BF704748BF52
:1003600020F8022B11F0804F18BF00F8012B7047C6
:10037000704770477047704700487047202D002035
:100380007546FFF7F9FFAE4605006946534620F073
:100390000700854618B020B5FFF726FFBDE82040CE
:1003A0004FF000064FF000074FF000084FF0000B31
:1003B00021F00701AC46ACE8C009ACE8C009ACE8E4
:1003C000C009ACE8C0098D46704710B50446AFF3CC
:1003D00000802046BDE81040FFF7F1BE10B540F2A6
:1003E00044620249024800F0B5F910BD181400201B
:1003F00000F0030810B50B480068401C094908606C
:100400000846006844F62061884209D30846054939
:10041000086000BF00220121034800F0A5FF00BFD3
:1004200010BD000028000020000C014010B500BFE6
:1004300001221146034800F097FF00BF0020024947
:10044000086010BD000C01402800002000BFFEE73E
:10045000F0B502460C46FF21FF2509E012F8016BBA
:1004600086EA0103084EF65C86EA0501074EF55C54
:10047000261EA4F10107BCB2F0D108464FF6FF7664
:1004800006EA00202843F0BD383C0008383D00084B
:10049000F0B505460C46A01E2E5C4FF6FF7000EA34
:1004A0000626601E285C0643A01E81B22846FFF780
:1004B000CFFF0746BE4201D10120F0BD0020FCE77E
:1004C00070B500BFD52002F0AFFF00BF0021084685
:1004D00002F0DEFC002416E000250DE0002002F012
:1004E000D9FF002002F0D6FF002002F0D3FF002049
:1004F00002F0D0FF681C85B2142DEFDB002002F063
:10050000C9FF601C84B2A02CE6DB70BD10B50248A8
:1005100000F094FA10BD0000D413002070470000D2
:100520002DE9F84F81460F46904630A000680090B4
:1005300000BFD52002F078FF00BFB9F1A00F01D8AD
:10054000A02F01D9BDE8F88FC9F1A0004008032110
:10055000B0FBF1F000F0FF0AC7F1A00007EB50007C
:1005600000F0FF0B4FEAD90600243BE0ABEB0400A0
:10057000C1B2504602F08CFC00252CE004FB065171
:1005800018F80110C943C1F381111DF8010002F0F0
:1005900081FF04FB065118F80110C943C1F3011192
:1005A0001DF8010002F076FF04FB065118F8011057
:1005B000C943C1F381011DF8010002F06BFF04FB88
:1005C000065118F80120032191431DF8010002F0A3
:1005D00061FF681CC5B2B542D0D3002002F05AFFBB
:1005E000601CC4B2BC42C1D300BFABE7000FF0FF38
:1005F0000021074AD1610749096941F00401054A10
:1006000011611146096941F0400111617047000014
:1006100060010020002002400021074AD161074903
:10062000096941F00201054A1161114648610969F1
:1006300041F040011161704760010020002002403C
:100640000022054BDA61054A126942F00102034BB0
:100650001A61018070470000600100200020024004
:1006600000201E49C96801F0100139B11C49C9694F
:1006700041F002011A4AD16140F010001749C968DF
:1006800001F0040139B11649C96941F00101144A68
:10069000D16140F004001149C96901F0010169B15B
:1006A0000F49C96941F004010D4AD16100BF0B49EE
:1006B000C96921F00101094AD16100BF00BF40F2C0
:1006C0000111884206D10549C96921F00101034A97
:1006D000D16101E00149C86000BF704700200240BD
:1006E0006001002070B5044600F044FE054609E0B4
:1006F000601C38B124B100F03DFE401BA04201D97E
:10070000032070BD1248C06800F001000028EFD13E
:100710000F48C06800F0200020B100BF20200C4925
:10072000C86000BF0A48C06800F0100048B9084817
:10073000C06900F0010020B90548C06800F004005D
:1007400018B1FFF78DFF0120DBE70020D9E700009B
:10075000002002402DE9F74F88B005469046A5F1EC
:100760000060079007984FEAD02A4FF0006000EB36
:10077000CA26A81B06904FEA4807059506983844F4
:100780004FEAD02B4FF00009002000900698384423
:10079000C0F30A0008B10BF1010BB5F1006F03D3F0
:1007A000E8192549884203D301200BB0BDE8F08F3A
:1007B000B6F1006F02D32048864201D30120F4E74E
:1007C00000F008FC0598C11906F5006081422ED39F
:1007D000002414E000200190039601200490694653
:1007E00001A800F03DFB8146B9F1000F03D000F0F5
:1007F0008FFB4846D9E706F50066601C84B25C456D
:10080000E8D3002410E0099830F814C005EB440147
:1008100062460023012000F085FB8146B9F1000FFC
:1008200000D003E0601C84B24445ECDB00BF00F064
:100830006FFB4846B9E700000000040801460022AB
:1008400091F82100022808D00420886300BF00200E
:1008500081F8200000BF012070470868006820F080
:100860000E000B6818600868006820F001000B6833
:10087000186091F8403001209840CB6B58600120FF
:1008800081F8210000BF002081F8200000BF104641
:10089000E2E7000070B50446002594F82100022824
:1008A00003D00420A0630125C1E02068006820F087
:1008B0000E00216808602068006820F001002168AF
:1008C00008605C492068884252D95A4978392068C2
:1008D000884201D1012047E05649643920688842A6
:1008E00001D1102040E0534950392068884201D19D
:1008F000801539E04F493C392068884201D1801485
:1009000032E04C4928392068884202D14FF48030C7
:100910002AE0484914392068884202D14FF48010F7
:1009200022E044492068884201D140041CE0424949
:100930002068884201D1012016E03F491431206827
:10094000884201D110200FE03B49283120688842BD
:1009500001D1801508E038493C312068884201D136
:10096000801401E04FF480303349091F086051E0E2
:10097000304978392068884201D1012047E02D496B
:1009800064392068884201D1102040E0294950395B
:100990002068884201D1801539E026493C39206819
:1009A000884201D1801432E02249283920688842E7
:1009B00002D14FF480302AE01E4914392068884261
:1009C00002D14FF4801022E01A492068884201D1F8
:1009D00040041CE018492068884201D1012016E03B
:1009E000154914312068884201D110200FE01249C6
:1009F00028312068884201D1801508E00E493C3139
:100A00002068884201D1801401E04FF48030094908
:100A100080394860012084F8210000BF002084F85C
:100A2000200000BF606B10B12046616B88472846EC
:100A300070BD0000800002400804024070B504460A
:100A4000E06B05682068066894F840100420884030
:100A50002840002875D006F004000028FAD020684D
:100A6000006800F0200028B92068006820F0040029
:100A700021680860D5492068884254D9D34978391B
:100A80002068884201D1042049E0D04964392068B7
:100A9000884201D1402042E0CC4950392068884248
:100AA00001D100153BE0C9493C392068884202D198
:100AB0004FF4804033E0C54928392068884202D18C
:100AC0004FF480202BE0C14914392068884202D1BC
:100AD0004FF4800023E0BD492068884201D1C00462
:100AE0001DE0BB492068884201D1042017E0B849C5
:100AF00014312068884201D1402010E0B4492831E7
:100B00002068884201D1001509E0B1493C312068D4
:100B1000884202D14FF4804001E04FF48020AC497C
:100B2000091F086054E0A94978392068884201D13A
:100B300004204AE0A54964392068884202D1402057
:100B400043E04CE0A14950392068884201D10015AA
:100B50003BE09E493C392068884202D14FF48040F6
:100B600033E09A4928392068884202D14FF4802026
:100B70002BE0964914392068884202D14FF4800056
:100B800023E092492068884201D1C0041DE09049C9
:100B90002068884201D1042017E08D491431206873
:100BA000884201D1402010E08949283120688842DC
:100BB00001D1001509E086493C312068884202D104
:100BC0004FF4804001E04FF4802080498039486034
:100BD000E06A002802D02046E16A8847F4E094F8F1
:100BE0004010022088402840002871D006F0020002
:100BF0000028FAD02068006800F0200040B9206882
:100C0000006820F00A0021680860012084F82100B3
:100C10006E492068884254D96C49783920688842E6
:100C200001D1022049E0694964392068884201D134
:100C3000202042E0654950392068884201D14015A2
:100C40003BE062493C392068884202D14FF40050B1
:100C500033E05E4928392068884202D14FF40030E1
:100C60002BE05A4914392068884202D14FF4001011
:100C700023E056492068884201D180041DE0544990
:100C80002068884201D1022017E0514914312068C0
:100C9000884201D1202010E04D4928312068884247
:100CA00001D1401509E04A493C312068884202D10F
:100CB0004FF4005001E04FF400304549091F08602F
:100CC00054E0424978392068884202D102204AE043
:100CD00057E03E4964392068884201D1202042E033
:100CE0003A4950392068884201D140153BE03749E4
:100CF0003C392068884202D14FF4005033E0334938
:100D000028392068884202D14FF400302BE02F4967
:100D100014392068884202D14FF4001023E02B4997
:100D20002068884201D180041DE02949206888425A
:100D300001D1022017E0264914312068884201D1F0
:100D4000202010E0224928312068884201D1401536
:100D500009E01F493C312068884202D14FF400501D
:100D600001E04FF4003019498039486000BF00208D
:100D700084F8200000BFA06A30B32046A16A8847EB
:100D800022E094F84010082088402840E0B106F0A6
:100D90000800C8B12068006820F00E0021680860D3
:100DA00094F8401001208840E16B48600120A06366
:100DB00084F8210000BF002084F8200000BF206BD1
:100DC00010B12046216B884770BD000080000240B2
:100DD000080402400146002209B9012070471E4B59
:100DE000086898420BD21D4B0868C01A1423B0FB48
:100DF000F3F08000086419480838C8630AE0164B0D
:100E00000868C01A1423B0FBF3F08000086412488D
:100E10000838C863022081F821000868026843F698
:100E2000F0708243D1E901031843CB6818430B6982
:100E300018434B6918438B691843CB691843024325
:100E40000868026000208863012081F821000020EA
:100E500081F8200000BFC1E70804024008000240FA
:100E60002DE9F04104460E460127002500BF264823
:100E7000007E012802D10220BDE8F0810120224934
:100E8000087600BF2068022813D14CF25030FFF7DB
:100E900029FC90BB0120FFF7ABFB4CF25030FFF771
:100EA00021FC07461948006920F004001749086131
:100EB00023E04CF25030FFF715FCF0B94FF0FF3053
:100EC0003060A56812E02846FFF7A6FB4CF25030D0
:100ED000FFF708FC07460D48006920F002000B49A7
:100EE00008610FB1356007E005F50065D4E902102F
:100EF00001EBC020A842E6D800BF00BF0020024995
:100F0000087600BF3846B7E76001002000200240A5
:100F10000348006940F080000149086100207047E3
:100F2000002002402DE9FE4F05468B4617469846A5
:100F3000012600240020029000BF2448007E0128E2
:100F400002D10220BDE8FE8F01202049087600BFB3
:100F50004CF25030FFF7C6FB064686BB012D02D18E
:100F60000120029006E0022D02D10220029001E051
:100F70000420029000241EE02201B946C2464846E1
:100F80005146FFF744F980B20190022000FB04B003
:100F900000900199FFF754FB4CF25030FFF7A2FB91
:100FA00006460B48006920F001000949086106B1B6
:100FB00004E0601CC4B202988442DDDB00BF00BFC5
:100FC00000200249087600BF3046BBE760010020E0
:100FD0000020024000200849096901F0800151B158
:100FE0000649054A5160064951601146096901F0F8
:100FF000800101B1012070470020024023016745B4
:10100000AB89EFCD2DE9F847024600239C467BE1F2
:101010004FF0010808FA03F4D1F8008008EA040050
:10102000A0427DD1DFF8F4A2D1F80480A8EB0A0930
:10103000D0453AD014DCB8F1030F50D009DCB8F138
:10104000000F31D0B8F1010F1CD0B8F1020F49D117
:1010500020E0B8F1110F18D0B8F1120F42D11EE004
:10106000B9F5881F25D006DCB9F5803F20D0B9F549
:10107000801F37D11AE0B9F5001F18D0B9F5041F49
:1010800030D117E0D1F80CC02DE0D1F80C8008F178
:10109000040C28E0D1F80C8008F1080C23E0D1F80A
:1010A0000C8008F10C0C1EE000BF00BF00BF00BFA9
:1010B00000BF00BFD1F80880B8F1000F02D14FF097
:1010C000040C0BE0D1F80880B8F1010F03D14FF008
:1010D000080C146102E04FF0080C546103E04FF07B
:1010E000000C00E000BF00BFFF2801D8904601E0DF
:1010F00002F104084646FF2802D84FEA830803E0BD
:10110000A3F108084FEA88084746D6F800804FF058
:101110000F0909FA07F928EA09080CFA07F900E0AB
:101120007AE048EA0908C6F80080D1F8048008F09F
:101130008058B8F1805F6FD100BFDFF8E481D8F844
:10114000188048F00108DFF8D891C9F81880C8461F
:10115000D8F8188008F00108CDF8008000BF00BF63
:101160004FEAB9384FEA930958F829504FEA837883
:101170004FEA18794FF00F0808FA09F825EA080530
:10118000DFF8A081424502D14FF0000824E0DFF8EB
:101190009881424502D14FF001081DE0DFF88C81B3
:1011A000424502D14FF0020816E0DFF88481424543
:1011B00002D14FF003080FE0DFF87881424502D1F9
:1011C0004FF0040808E0DFF87081424502D14FF08B
:1011D000050801E04FF006084FEA83794FEA1979D4
:1011E00008FA09F848EA0505DFF850814FEA930943
:1011F00048F82950D1F8048008F48018B8F5801F09
:101200000BD1DFF83C81D8F8008048EA0008DFF80D
:101210003091C9F800800AE075E0DFF82481D8F841
:10122000008028EA0008DFF81891C9F80080D1F89A
:10123000048008F40018B8F5001F0ED1DFF8008113
:1012400008F10408D8F8008048EA0008DFF8F090B8
:1012500009F10409C9F800800DE0DFF8E48008F125
:101260000408D8F8008028EA0008DFF8D49009F1D3
:101270000409C9F80080D1F8048008F40038B8F5F2
:10128000003F0ED1DFF8B880A8F10408D8F800803C
:1012900048EA0008DFF8A890A9F10409C9F800801D
:1012A0000DE0DFF89C80A8F10408D8F8008028EA57
:1012B0000008DFF88C90A9F10409C9F80080D1F882
:1012C000048008F48038B8F5803F0ED1DFF87080D4
:1012D000A8F10808D8F8008048EA0008DFF8609014
:1012E000A9F10809C9F800800DE0DFF85480A8F1E1
:1012F0000808D8F8008028EA0008DFF84490A9F12F
:101300000809C9F800805B1CD1F8008028FA03F8AE
:10131000B8F1000F7FF47CAEBDE8F8870000111033
:101320000010024000080140000C01400010014084
:101330000014014000180140001C01400800014059
:1013400008040140024693680B400BB1012000E005
:101350000020704710B5C26821EA020302EA0104C6
:1013600043EA0443036110BD0AB1016101E00B04CB
:1013700003617047014800687047000018000020B2
:101380000348006803490978084401490860704728
:10139000180000202000002010B50848006840F028
:1013A000100006490860032000F080F80F2000F0CC
:1013B00007F800F02BF8002010BD000000200240CC
:1013C00070B504460E4800784FF47A71B1FBF0F026
:1013D0000C490968B1FBF0F5284600F0F3FB08B1B1
:1013E000012070BD102C07D200222146501E00F0B3
:1013F0001EF80548046001E00120F2E70020F0E754
:1014000020000020080000201C000020704701463A
:101410000846002809DB00F01F0301229A40430917
:101420009B0003F1E023C3F8002100BF70472DE9C2
:10143000F05F80460D461646002702F05FF807462B
:1014400039462A46334601F00700C0F1070ABAF1CF
:10145000040F02D94FF0040A01E0C0F1070AD14697
:1014600000F1040ABAF1070F02D24FF0000A01E0BE
:10147000A0F1030AD4464FF0010A0AFA09FAAAF1C8
:10148000010A0AEA020A0AFA0CFA4FF0010B0BFAF7
:101490000CFBABF1010B0BEA030B4AEA0B042146F0
:1014A000404602F033F8BDE8F09F000000BF00F0B6
:1014B0000702064B19684FF6FF031940044B0B4314
:1014C00043EA0221014B196000BF70470CED00E0B8
:1014D0000000FA0500BF00BF00BF00BF00BFBFF3A0
:1014E0004F8F00BF00BF00BF0948006800F4E060F4
:1014F00008490843001D0649086000BF00BF00BF3F
:10150000BFF34F8F00BF00BF00BF00BF00BFFDE7AC
:101510000CED00E00000FA0570B504460D460CB96C
:10152000012070BD5A48006800F00700A8420ED2A2
:101530005748006820F007002843554908600846CE
:10154000006800F00700A84201D00120E9E72078F8
:1015500000F0020002281DD1207800F004000428C9
:1015600005D14C48406840F4E0604A494860207822
:1015700000F00800082805D14648406840F4605053
:10158000444948604348406820F0F000A16808439F
:1015900040494860207800F0010078B36068012875
:1015A00006D13C48006800F4003090B90120B8E74B
:1015B0006068022806D13748006800F0007040B922
:1015C0000120AEE73348006800F0020008B90120AE
:1015D000A7E73048406820F00300616808432D49C0
:1015E0004860FFF7C7FE064609E0FFF7C3FE801B11
:1015F00041F28831884202D9032092E707E025486A
:10160000406800F00C006168B0EB810FEDD120481C
:10161000006800F00700A8420ED91D48006820F0BD
:10162000070028431A4908600846006800F00700D0
:10163000A84201D0012074E7207800F004000428BB
:1016400007D11448406820F4E060E168084311497C
:101650004860207800F00800082808D10D4840684C
:1016600020F46050216940EAC1000A49486000F056
:101670003FF808494968C1F30311074A515CC84063
:101680000649086006480068FFF79AFE002048E710
:1016900000200240001002407A3A000808000020B2
:1016A0001C0000200148006870470000080000206E
:1016B00000B5FFF7F7FF04494968C1F30221034A67
:1016C000515CC84000BD0000001002408A3A00088A
:1016D00000B5FFF7E7FF04494968C1F3C221034A97
:1016E000515CC84000BD0000001002408A3A00086A
:1016F00070B500210022002400230020134D6968EA
:1017000001F00C05F5B1042D02D0082D19D101E02E
:101710000F4819E00F4DC1F38346AB5D01F48035EE
:1017200055B10A4D6D68C5F340450B4E725D084DCD
:101730005D43B5FBF2F402E0084D03FB05F42046DF
:1017400002E000BF024800BF00BF70BD00100240B1
:1017500000127A00923A0008A23A000800093D00FF
:10176000F8B504460CB90120F8BD207800F001005E
:10177000002878D0F848406800F00C0004280CD00D
:10178000F548406800F00C00082811D1F248406884
:1017900000F48030B0F5803F0AD1EF48006800F4D3
:1017A000003000285FD0606800285CD10120DBE7B2
:1017B00000BF6068B0F5803F06D1E748006840F49C
:1017C0008030E549086028E0606858B9E248006860
:1017D00020F48030E04908600846006820F480204A
:1017E00008601AE06068B0F5A02F0BD1DA480068F5
:1017F00040F48020D84908600846006840F48030F2
:1018000008600AE0D448006820F48030D2490860BB
:101810000846006820F48020086000BF606888B136
:10182000FFF7A8FD054606E0FFF7A4FD401B64286E
:1018300001D9032098E7C848006800F40030002868
:10184000F2D010E0FFF796FD054606E0FFF792FDA7
:10185000401B642801D9032086E7BF48006800F4D4
:1018600000300028F2D1207800F00200022857D181
:10187000B948406800F00C0050B1B748406800F02B
:101880000C00082818D1B448406800F4803098B99A
:10189000B148006800F0020020B12069012801D0A1
:1018A000012061E7AC48006820F0F800616940EA77
:1018B000C100A949086033E02069E8B10120A749C7
:1018C0000860FFF757FD054606E0FFF753FD401B94
:1018D000022801D9032047E79F48006800F0020072
:1018E0000028F2D09C48006820F0F800616940EAC6
:1018F000C1009949086013E0002098490860FFF78B
:1019000039FD054606E0FFF735FD401B022801D9E9
:10191000032029E79048006800F002000028F2D177
:10192000207800F0080008282DD1A069B8B1012066
:101930008B490860FFF71EFD054606E0FFF71AFD1C
:10194000401B022801D903200EE78348406A00F0BB
:1019500002000028F2D0012001F058F813E0002026
:101960007F490860FFF706FD054606E0FFF702FD28
:10197000401B022801D90320F6E67748406A00F0B0
:1019800002000028F2D1207800F00400042873D16E
:1019900000277148C06900F0805070B900BF6E48E0
:1019A000C06940F080506C49C8610846C06900F0C9
:1019B0008050009000BF00BF01276A48006800F413
:1019C0008070B0B96748006840F48070654908606D
:1019D000FFF7D0FC054606E0FFF7CCFC401B64286F
:1019E00001D90320C0E65F48006800F48070002839
:1019F000F2D000BFE068012806D15748006A40F0E5
:101A000001005549086227E0E06858B95248006A69
:101A100020F00100504908620846006A20F00400E6
:101A2000086219E0E06805280BD14B48006A40F0D5
:101A30000400494908620846006A40F00100086253
:101A40000AE04548006A20F0010043490862084660
:101A5000006A20F00400086200BFE068A0B1FFF750
:101A600089FC054609E0FFF785FC401B41F28831FF
:101A7000884202D9032077E622E03748006A00F066
:101A800002000028EFD012E0FFF774FC054608E0E2
:101A9000FFF770FC401B41F28831884201D90320D6
:101AA00062E62D48006A00F002000028F0D1012F04
:101AB00005D12948C06920F080502749C86100BF7E
:101AC000E069C8B32448406800F00C00082860D0E2
:101AD000E069022848D1002020490866FFF74AFC47
:101AE000054606E0FFF746FC401B022801D903200B
:101AF0003AE61948006800F000700028F2D1206A28
:101B0000B0F5803F07D11448406820F40030A16848
:101B1000084311494860D4E9080108430E4949685F
:101B200021F4741108430C49486001200B490866F0
:101B3000FFF720FC054607E03DE0FFF71BFC401BDC
:101B4000022801D903200FE60348006800F0007066
:101B50000028F2D02FE000000010024000004242B6
:101B60008004424200700040002014490866FFF7DC
:101B700001FC054606E0FFF7FDFB401B022801D9EA
:101B80000320F1E50E48006800F000700028F2D153
:101B900011E0E069012800D1E6E50948466806F44D
:101BA0008031206A814204D106F47011606A81425A
:101BB00001D00120D8E50020D6E500000000424217
:101BC0000010024070B504462546681EB0F1807FC3
:101BD00001D301200FE0681E4FF0E02148610F2182
:101BE0004FF0FF3001F092FC00204FF0E0218861BF
:101BF00007200861002070BD10B504460CB9012013
:101C000010BD94F83D0028B9002084F83C0020461F
:101C100000F025F8022084F83D00211D206801F025
:101C20008BF9012084F8460000BF84F83E000121B2
:101C30003F200155402001554120015500BF00BF04
:101C4000012084F8420043200155442001554520DD
:101C5000015500BF012084F83D000020D0E7704707
:101C6000014691F83D00012801D001207047022073
:101C700081F83D000868C06840F001000B68D8603A
:101C8000164B0868984213D0154B086898420FD03D
:101C90000868B0F1804F0BD0124B0868984207D00B
:101CA000114B0868984203D0104B086898420CD139
:101CB0000868806800F00702062A0CD008680068EF
:101CC00040F001000B68186005E00868006840F00B
:101CD00001000B6818600020C8E70000002C0140DC
:101CE000003401400004004000080040000C0040A7
:101CF000F8B504460E46174694F8420020282ED127
:101D000006B10FB90120F8BD0120206300206063F7
:101D10003A463146204601F0B1FA0546EDB9206B4E
:101D2000012819D100BF00200090206800680090B1
:101D300020684068009000BF00BF00BF00BF21685E
:101D40000C3151E8001F41F0100021680C3141E8CE
:101D50000002002AF3D100E001252846D3E7022043
:101D6000D1E7000070B504460D4607492068884257
:101D700008D101200549087041F27002491C04484D
:101D8000FFF7B6FF70BD00000044004010030020C4
:101D90008C130020704700002DE9F84F044620689E
:101DA00005682068C668206847694FF00009CA4680
:101DB00005F00F09B9F1000F0AD105F0200038B184
:101DC00006F0200020B1204601F05CF9BDE8F88F54
:101DD000B9F1000F7BD007F0010018B906F490703C
:101DE000002874D005F0010030B106F4807018B1FD
:101DF000606C40F00100606405F0040030B107F051
:101E0000010018B1606C40F00200606405F002004F
:101E100030B107F0010018B1606C40F0040060645C
:101E200005F0080048B106F0200010B907F00100E5
:101E300018B1606C40F008006064606C002845D008
:101E400005F0200028B106F0200010B1204601F076
:101E500019F920684069C0F3801A606C00F008002E
:101E600010B9BAF1000F2CD0204601F0C5F8206857
:101E7000406900F0400000B300BF00BF216814318A
:101E800051E8001F21F040002168143141E80002B0
:101E9000002AF3D100BFE06B50B17748E16B486393
:101EA000E06BFEF7F7FC88B1E06B416B88470DE013
:101EB0002046FFF76FFF09E009E02046FFF76AFFC1
:101EC00004E02046FFF766FF002060647EE7206B99
:101ED000012877D105F01000002873D006F010001B
:101EE0000028FAD000BF0020009020680068009011
:101EF00020684068009000BF00BF2068406900F083
:101F0000400000285FD0E06B006840681FFA80F84E
:101F1000B8F1000F55D0A08D404552DDA4F82E80B9
:101F2000E06B8069202843D000BF00BF21680C31DE
:101F300051E8001F21F4807021680C3141E8000253
:101F4000002AF3D100BF00BF00BF2168143151E85F
:101F5000001F21F001002168143141E80002002A2D
:101F6000F3D100BF00BF00BF2168143151E8001F4A
:101F700021F040002168143141E80002002AF3D129
:101F800000BF202084F842000020206300BF00BF73
:101F900021680C3151E8001F21F0100021680C313C
:101FA00041E80002002AF3D100BFE06BFEF746FCD7
:101FB00002206063A08DE28D801A81B22046FFF777
:101FC000D1FE03E742E0A08DE18D401A1FFA80F8B0
:101FD000E08DD0B3B8F1000F37D000BF00BF21684B
:101FE0000C3151E8001F21F4907021680C3141E858
:101FF0000002002AF3D100BF00BF00BF21681431E6
:1020000051E8001F21F001002168143141E800026D
:10201000002AF3D100BF202084F842000020206372
:1020200000BF00BF21680C3151E8001F21F01000F3
:1020300021680C3141E80002002AF3D100BF0220E0
:10204000606341462046FFF78DFEBFE605F0800045
:1020500030B106F0800018B1204601F02FF9B5E646
:1020600005F0400030B106F0400018B1204600F005
:10207000F9FFABE600BFA9E6E52F000810B504465E
:102080000CB9012010BDA06900B100E000BF94F8B8
:10209000410028B9002084F84000204600F02AF8CA
:1020A000242084F841002068C06820F40050216892
:1020B000C860204601F064F82068006920F4904070
:1020C000216808612068406920F02A002168486181
:1020D0002068C06840F400502168C8600020606437
:1020E000202084F8410084F842000020606300BF93
:1020F000C8E7000010B586B0044628492068884229
:102100004AD100BF00BF2648806940F0040024493E
:1021100088610846806900F00400019000BF00BF9C
:1021200000BF00BF00BF0846806940F0040088611E
:102130000846806900F00400019000BF00BF00BFA6
:1021400000BF00BF0846806940F4804088610846AF
:10215000806900F48040019000BF00BF00BF4815B7
:10216000029002200390012004900320059002A910
:102170000C48FEF747FF4FF4806002900020039068
:1021800002A90848FEF73EFF2520FFF740F9032289
:1021900011462520FFF74BF906B010BD003801406D
:1021A000001002400008014070B504460D46164676
:1021B00094F8420020280BD105B10EB9012070BD62
:1021C0000020206332462946204601F057F8F6E702
:1021D0000220F4E710B504462049206888423BD12C
:1021E0001F48008800F4004088BB1D48008800F4A8
:1021F000804070B11B4800780A2803D0002018499D
:10220000088024E01648008840F400401449088003
:102210001DE0144800780D2806D11148008840F4CC
:1022200080400F49088012E00E4800780C49098868
:10223000C1F30D010C4A505409480088401C08495C
:10224000088008460088C72801DD00200880012298
:1022500004490648FFF7A8FF10BD00000038014000
:10226000140000201600002050000020180100205B
:102270002DE9F84F04460E46174699464FF0000ADE
:1022800094F84100202850D106B117B90120BDE8CB
:10229000F88F00206064212084F84100FFF76AF87D
:1022A0008246A784E784A068B0F5805F04D12069E6
:1022B00010B90025B04602E035464FF000081EE098
:1022C0005346002280212046CDF8009001F026F8E8
:1022D00020B1202084F841000320D8E745B9B8F8A0
:1022E0000000C0F308002168486008F1020803E01C
:1022F0002878216848606D1CE08C401EE084E08CEA
:102300000028DDD15346002240212046CDF8009020
:1023100001F004F820B1202084F841000320B6E742
:10232000202084F841000020B1E70220AFE7704789
:1023300000BFFEE708B5434A811A904241D009DC4C
:102340004149014481B1B1F5806F1CD0B1F5006FF6
:1023500074D127E0B1F5806F42D0B1F5006F4ED057
:10236000B1F5406F6AD159E000BF3849896941F041
:102370000401364A91611146896901F00401009116
:1023800000BF00BF5BE000BF3049896941F0080130
:102390002E4A91611146896901F00801009100BF40
:1023A00000BF4CE000BF2949896941F01001274A6C
:1023B00091611146896901F01001009100BF00BFD1
:1023C0003DE000BF2149896941F020011F4A916128
:1023D0001146896901F02001009100BF00BF2EE085
:1023E00000BF1A49896941F04001184A91611146BC
:1023F000896901F04001009100BF00BF1FE000BFEC
:102400001249896941F08001104A91611146896938
:1024100001F08001009100BF00BF10E000BF0B4938
:10242000896941F48071094A91611146896901F411
:102430008071009100BF00BF01E0FFE700BF00BF57
:1024400008BD00000014014000F8FEBF001002406B
:1024500010B586B000BF2F48806940F001002D49BB
:1024600088610846806900F00100019000BF00BF4C
:1024700000BF2949486820F0E06040F000704860E3
:1024800000BF0020029003900490059000243DE0DE
:1024900004EB4401214A02EB81014868FFF74AFF3F
:1024A00004EB44001D4931F8200002900020039005
:1024B00004900320059004EB4401184A02EB8101CB
:1024C000486802A9FEF79EFD04EB440101EBC4013C
:1024D000134A02EB810023460022124901F086F9DB
:1024E00004EB440101EBC4010D4A02EB81000E4AEA
:1024F000032101F021F804EB440101EBC401084A77
:1025000002EB810001F0AEF9601CC4B2072CBFD30E
:1025100006B010BD0010024000000140E43B00087E
:10252000DC0100203D3800084D35000810B5044698
:10253000FDF77CFF0148047010BD0000040000207E
:1025400001490860704700002400002000B585B0F4
:1025500000BF1A48806940F00800184988610846A1
:10256000806900F00800009000BF00BF00BF08466F
:10257000806940F0400088610846806900F04000B2
:10258000009000BF00BF47F601400190012002907B
:1025900003900320049001A90948FEF733FD4FF48E
:1025A0007F4001900120029003900320049001A934
:1025B0000448FEF727FD05B000BD000000100240F2
:1025C000000C01400018014010B5E92000F02CFF7C
:1025D0002B2000F029FF242000F026FF812000F0AE
:1025E00023FFBE2000F020FFA42000F01DFFA62046
:1025F00000F01AFFC02000F017FFA32000F014FF26
:10260000D12000F011FFD52000F00EFFDA2000F0FD
:102610000BFFF42000F008FF252000F005FFF62056
:1026200000F002FF5A2000F0FFFEF52000F0FCFE53
:10263000002000F0F9FEF72000F0F6FE9F2000F0E9
:10264000F3FEF82000F0F0FE892000F0EDFEAD2052
:1026500000F0EAFE402000F0E7FE502000F0E4FE2B
:10266000C42000F0E1FE902000F0DEFEFF2000F02C
:10267000DBFE842000F0D8FEF12000F0D5FE9F2084
:1026800000F0D2FE10BD000010B500BF0122910283
:102690000E48FEF769FE00BF0A2001F011F900BFE5
:1026A00000224FF480610948FEF75EFE00BF022061
:1026B00001F006F900BF012291020448FEF754FE22
:1026C00000BF962001F0FCF810BD0000000C014096
:1026D00008B5434A811A904241D009DC414901447E
:1026E00081B1B1F5806F1CD0B1F5006F74D127E0D6
:1026F000B1F5806F42D0B1F5006F4ED0B1F5406FAB
:102700006AD159E000BF3849896941F00401364A6D
:1027100091611146896901F00401009100BF00BF79
:102720005BE000BF3049896941F008012E4A9161A0
:102730001146896901F00801009100BF00BF4CE01B
:1027400000BF2949896941F01001274A916111466A
:10275000896901F01001009100BF00BF3DE000BF9A
:102760002149896941F020011F4A91611146896917
:1027700001F02001009100BF00BF2EE000BF1A4908
:10278000896941F04001184A91611146896901F057
:102790004001009100BF00BF1FE000BF12498969DE
:1027A00041F08001104A91611146896901F0800170
:1027B000009100BF00BF10E000BF0B49896941F4E0
:1027C0008071094A91611146896901F48071009113
:1027D00000BF00BF01E0FFE700BF00BF08BD000071
:1027E0000014014000F8FEBF001002401FB5002495
:1027F00047E0274901EB04110868FFF769FF244807
:1028000000EB04108088009001200190204800EB2C
:102810000410806803901E4800EB0410C06802900A
:102820001B4901EB041108686946FEF7EBFB184BE6
:1028300003EB0413DA79164B03EB04139988144B5A
:1028400003EB04131868FEF78FFD114800EB04102A
:10285000807950B90E4800EB0410C07908B9012006
:1028600000E000200B49085509E0094800EB04107E
:10287000C079012800D100E0002006490855601CFD
:10288000C4B2142CB5DB0121002000F06FF81FBD8D
:10289000A43A00088001002070B50446142C00DB27
:1028A00070BD0C4800EB0410807908B9012500E0E8
:1028B0000025084A02EB04129188064A02EB041232
:1028C00010682A46FEF750FD00200349085500BF56
:1028D000E6E70000A43A00088001002070B5044635
:1028E000142C00DB70BD0C4800EB0410807908B993
:1028F000002500E00125084A02EB04129188064AEF
:1029000002EB041210682A46FEF72EFD012003494F
:10291000085500BFE6E70000A43A00088001002047
:102920002DE9F0410446E0780006A17840EA014034
:10293000617840EA0120217840EA01060025012162
:10294000002000F013F801250CE00120A8403040E1
:1029500008B1012000E000200746E8B2394600F047
:1029600005F86D1C142DF0D3BDE8F08170B5054657
:102970000C46012C03D12846FFF7B0FF02E02846A1
:10298000FFF78AFF70BD000010B5044AD2F8841C1E
:10299000D2F8800CFDF7C4FD10BD00001814002013
:1029A00010B5FFF7D3FD00BF012211460548FEF721
:1029B000DBFC00BFFFF768FEFFF706FEFDF780FDBA
:1029C00010BD0000000C014000BFFEE700BFFEE7A5
:1029D0007047000006480078401C0549087008460A
:1029E000007918B108464079401C487170470000D2
:1029F0003400002000200449887108714871C871B2
:102A000001204880704700003400002008B50849C4
:102A10000968C9084FF47A72B1FBF2F141430091A1
:102A200000BF00BF00994A1E00920029F9D108BDDD
:102A30000800002000B585B000BF00BF594880697C
:102A400040F00400574988610846806900F004009E
:102A5000009000BF00BF00BF00BF00BF08468069F4
:102A600040F0040088610846806900F0040000908E
:102A700000BF00BF00BF00BF00BF0846806940F034
:102A8000040088610846806900F00400009000BFDF
:102A900000BF00BF00BF00BF0846C06940F400305F
:102AA000C8610846C06900F40030009000BF00BF54
:102AB00000BF00BF0846406940F001004861084679
:102AC000406900F00100009000BF00BF00200190AD
:102AD00002900390049004200190022002900120B3
:102AE00003900320049001A92F48FEF78BFA0820D9
:102AF00001900020029001A92B48FEF783FA0220E2
:102B000001900120029001A92748FEF77BFA27488F
:102B10002749086000204860002125488160802105
:102B2000C16000210161416181614FF44051C16187
:102B3000FEF750F900BF1E481E49C86308461C49ED
:102B4000486200BF1020FEF762FC002211461020F0
:102B5000FEF76DFC184817490860184848600021C6
:102B600014488160C160016181610C2141610021D3
:102B7000C161FFF783FA2620FEF749FC00220121FC
:102B80002620FEF754FC00BF012202210648FEF772
:102B9000EBFB00BF41F2700209490648FFF7A8F8B5
:102BA00005B000BD00100240000801406C0002406A
:102BB000D41300208C1300200044004060AE0A00B3
:102BC0001103002010B504460CB155480470554857
:102BD0000078002872D000205249087041F270013C
:102BE0005048401CFDF754FC012854D100204E49A8
:102BF00008604FF448624B49491C4C48FDF71AFBEA
:102C00004B494C4802680A604068486008460079B1
:102C1000892834D108464079452830D14FF448629C
:102C200042494548FDF74BFB414840784049097807
:102C300040EA01204049C1F8800C3D48C0783C4939
:102C4000897840EA01203C49C1F8840CFDF7C6FBB5
:102C5000FDF7ECFBFDF734FCFFF796FE4FF4FA703E
:102C600000F02EFE4FF4FA7000F02AFE4FF4FA70D6
:102C700000F026FE4FF4FA7000F022FE16E02F4915
:102C80002848D0F8810C08600846FFF749FE27481D
:102C900000F0B2F80AE024480068401C22490860AD
:102CA00008460068032801D300200860002024495A
:102CB000887108714871C871012048802048408897
:102CC00010B91F48807998B11548007838B1144878
:102CD0000178002000F07AF80020114908701848A7
:102CE0000078372804DD0E480178012000F06EF8E6
:102CF00013484079282808DD0120114988710020F7
:102D000048710846C079401CC8710D48C079052833
:102D100004DB05200A49C8710120488010BD00006D
:102D20003C000020100300204C000020A0200020C8
:102D300041000020910F0020181400203D000020C9
:102D4000340000202DE9FC4104460D4616460027BC
:102D500001208DF800008DF801408DF802508DF8AB
:102D6000036004216846FDF773FB074638128DF8AF
:102D70000400F8B28DF805000621684600F008F856
:102D8000002002494880BDE8FC810000340000209A
:102D900070B504460D4600BF002202210948FEF727
:102DA000E3FA00BFAAB24FF47A7321460648FFF750
:102DB0005FFA00BF012202210248FEF7D5FA00BFE8
:102DC00070BD0000000801408C13002070B504465F
:102DD0000D462A4621460320FFF7B4FF0020044990
:102DE00048800870012008710020487170BD000003
:102DF0003400002070470000F8B5064600BFD5201B
:102E000000F012FB00BF21A00068009000210846DE
:102E100000F03EF8002436E000252DE004EB8401AC
:102E200005EB8101715C6A4602EB9111087800F0B4
:102E300031FB04EB840105EB8101715CC1F30111ED
:102E40001DF8010000F026FB04EB840105EB810175
:102E5000715CC1F381011DF8010000F01BFB04EB64
:102E6000840105EB8101715C01F003011DF8010093
:102E700000F010FB681C85B2142DCFDB002000F0A1
:102E800009FB601C84B2A02CC6DBF8BD000FF0FF6C
:102E900070B504460D4604F12500C4B204F00F00DD
:102EA00000F0C2FAC4F3021141F0100000F0BCFAC5
:102EB00005F00F0141F0600000F0B6FA702141EA20
:102EC000151000F0B1FA70BD10B5FEF759FA10BD3B
:102ED0007047000010B514480068006900F0010058
:102EE00000B312480068401C10490860084600689A
:102EF000C821B0FBF1F201FB120010B901200C490E
:102F0000087000F0C9FC00BF01210A48FEF722FA50
:102F100000BFFDF76FFAFFF75DFD6FF0010002499A
:102F20000968086110BD0000940100200000002025
:102F3000060000200008014010B50268244B9842AA
:102F40000ED0244B98420BD0B0F1804F08D0224BCA
:102F5000984205D0214B984202D0214B984203D190
:102F600022F070024B681A43194B98420ED0194B4D
:102F700098420BD0B0F1804F08D0174B984205D043
:102F8000164B984202D0164B984203D122F440725D
:102F9000CB681A4322F080034C6943EA04020260C2
:102FA0008B68C3620B688362094B984202D0094B5D
:102FB000984201D10B69036301234361036903F064
:102FC00001031BB1036923F00103036110BD00007D
:102FD000002C014000340140000400400008004083
:102FE000000C004070B505466C6A0020E085E08466
:102FF0002046FEF7CFFE70BD00BF00BF02680C3256
:1030000052E8002F22F4907102680C3242E800135B
:10301000002BF3D100BF00BF00BF0268143252E89A
:10302000002F22F001010268143242E80013002B45
:10303000F3D100BF016B01290ED100BF00BF0268B0
:103040000C3252E8002F22F0100102680C3242E8E4
:103050000013002BF3D100BF202180F84210002183
:103060000163704710B504462068C06820F0400036
:103070002168C860202084F841002046FFF757F9F6
:10308000002010BDF8B5044694F84200222875D1FE
:10309000A068B0F5805F0CD1206950B90025A66A00
:1030A00020684068C0F308003080A06A801CA062DD
:1030B00015E0A56A0026A068B0F5805F03D0A0687F
:1030C00028B9206918B920684068287004E0206891
:1030D000406800F07F002870A06A401CA062E08D6C
:1030E000401E80B2E085002846D12068C06820F0EC
:1030F00020002168C8602068C06820F480702168C2
:10310000C8602068406920F00100216848612020E3
:1031100084F8420000206063206B012826D1002043
:10312000206300BF00BF21680C3151E8001F21F06F
:10313000100021680C3141E80002002AF3D100BFE1
:103140002068006800F0100010280AD100BF00209D
:10315000009020680068009020684068009000BFE0
:1031600000BFA18D2046FEF7FDFD02E02046FFF7DF
:1031700031F80020F8BD01E00020FBE70220F9E76C
:1031800070B504462168096921F44051E268114391
:10319000226811612269A1681143626941EA02054E
:1031A0002168C96841F20C62914329432268D160C9
:1031B0002168496921F44071A26911432268516173
:1031C0002D4A2168914202D1FEF782FA01E0FEF712
:1031D0006FFA00EBC00101EB001162689200B1FBD5
:1031E000F2F100EBC00202EB001263689B00B2FB3D
:1031F000F3F26423B2FBF3F202EBC20303EB02121D
:10320000A1EB8201322202EB01116422B1FBF2F147
:1032100001F0F00100EBC00202EB001263689B00BA
:10322000B2FBF3F26423B2FBF3F201EB021200EB08
:10323000C00101EB001163689B00B1FBF3F100EBEF
:10324000C00303EB00136668B600B3FBF6F3642615
:10325000B3FBF6F303EBC30606EB0313A1EB830109
:10326000322303EB01116423B1FBF3F101F00F01F1
:1032700011442268916070BD0038014010B50346CA
:1032800099629A85DA8500205864222083F84200EA
:10329000186928B11868C06840F480701C68E06044
:1032A0001868406940F001001C6860611868C068D7
:1032B00040F020001C68E060002010BD014691F83D
:1032C0004100212828D18868B0F5805F0BD10869BA
:1032D00048B90A6A1088C0F308000B685860086A89
:1032E000801C086205E00B6A581C086218780B689D
:1032F0005860C88C401E80B2C88458B90868C0683D
:1033000020F080000B68D8600868C06840F040007A
:103310000B68D860002070470220FCE72DE9F843D5
:1033200004460D4617469846089E31E0701C70B35F
:10333000FEF720F8A0EB0800B04200D816B9032031
:10334000BDE8F8832068C06800F00400F8B1802D63
:103350001ED0402D1CD020680068C0F3C000B0B162
:1033600000BF00200090206800680090206840683E
:10337000009000BF00BF2046FFF73EFE08206064BB
:1033800000BF002084F8400000BF0120D8E7FFE71D
:10339000206800682840A84201D1012000E00020F8
:1033A000B842C3D00020CBE70021044A1268D1B252
:1033B00041EA0022014B1A60704700000C180140DE
:1033C00010B50248FEF7E8FC10BD0000180100200F
:1033D00010B50248FEF7E0FC10BD00008C13002081
:1033E00000BFFEE700B585B000BF00BF0C48806994
:1033F00040F004000A4988610846806900F0040032
:10340000009000BF00BF00BF012001900290039018
:103410000320049001A90348FDF7F4FD05B000BDA9
:10342000001002400008014010B5044600BF002211
:103430004FF480411648FDF797FF00BF00BF0122FF
:1034400011031348FDF790FF00BF2046FFF7ACFFC4
:1034500000BF00224FF400610D48FDF785FF00BF5B
:1034600000BF00224FF400510948FDF77DFF00BF67
:1034700000BF012251030648FDF776FF00BF00BFE1
:103480000122D1020248FDF76FFF00BF10BD00000E
:10349000000C014010B5044600BF012291031648FC
:1034A000FDF762FF00BF00BF012211031248FDF7C4
:1034B0005BFF00BF2046FFF777FF00BF00224FF4FD
:1034C00000610D48FDF750FF00BF00BF00224FF420
:1034D00000510948FDF748FF00BF00BF012251031A
:1034E0000548FDF741FF00BF00BF0122D10202489D
:1034F000FDF73AFF00BF10BD000C01400248006814
:10350000C0F30220704700000CED00E010B5002869
:1035100004DB0A07130E054A135406E00A07140ECB
:10352000034A00F00F031B1FD45410BD00E400E059
:1035300018ED00E000BF704708B1072900DB7047B5
:1035400000F10C0343F8212000BFF8E770B50446F2
:103550007CB10848006860B12579072D08D205EBD9
:103560004501054A02EB8101087A0249096888474A
:1035700000BF70BD24000020E43B000870B5044685
:1035800000BF2079A16888470546E07800F0070071
:10359000002802DD2088401C2080E078B5EBD01F99
:1035A00013D0E078C008401CE17860F3C501E170F9
:1035B000C1F3C20003280CDBE07865F3C710E070AC
:1035C000E07820F03800E07003E0E07820F0380088
:1035D000E070E07800F0070005287DD2DFE800F019
:1035E000032858AFDB00E078C0F38010E178B0EB3F
:1035F000D11F17D1A07820F0F000A07000BFE068C4
:1036000010B12046E168884700BF00202080A078E4
:1036100020F00F00401CA070E07820F00700401C54
:10362000E07004E0A07820F0F0008030A070DBE0D3
:10363000E078C0F38010E178B0EBD11F13D0A07810
:1036400020F0F0001030A07000BF206910B12046BB
:103650002169884700BF00202080E07820F0070023
:10366000801CE07013E02088C82810DDA07820F0CE
:10367000F0005030A07000BF206A10B12046216ACF
:10368000884700BFE07820F00700001DE070ABE045
:10369000E078C0F38010E178B0EBD11F25D1A0789D
:1036A00020F0F000A07000BFE06810B12046E16893
:1036B000884700BFA07800F00F000F2804DAA07838
:1036C000411C61F30300A07000BF606910B1204687
:1036D0006169884700BF00E081E000202080E07839
:1036E00020F00700C01CE07028E020883C2825DD81
:1036F000A07800F00F0001280BD1A07820F0F00096
:103700003030A07000BFA06910B12046A169884781
:1037100010E0A07800F00F0002280BD1A07820F074
:10372000F0004030A07000BFE06910B12046E169B0
:10373000884700BFE07820F00700E07054E0E078B0
:10374000C0F38010E178B0EBD11F1BD0A07820F03F
:10375000F0001030A07000BF206910B12046216930
:10376000884700BF20883C2807DA00202080E078C6
:1037700020F00700801CE0700CE0E07820F00700EB
:10378000E07007E020883C2804DDE07820F00700A6
:10379000401CE07028E0E078C0F38010E178B0EBE6
:1037A000D11F0BD1A07820F0F0006030A07000BFD6
:1037B000606A10B12046616A88470FE0A07820F067
:1037C000F0001030A07000BF206910B120462169C0
:1037D000884700BFE07820F00700E07004E0E07860
:1037E00020F00700E07000BF00BF70BD2DE9F04180
:1037F00004460D4616461F4604B10DB9BDE8F081DA
:103800002C212046FCF78DFDA07820F0F0008030C0
:10381000A070A5600EB9012000E00020E17860F3FF
:10382000C711E170E07866F38610E0702771E078E8
:1038300020F00700E07000BFE0E7000070B504462C
:1038400004EB4402064B33F8221004EB440203EB72
:1038500082025068FDF776FD0546284670BD0000DF
:10386000E43B0008014611B96FF0010070470948B8
:10387000026805E08A4202D14FF0FF30F6E7926A13
:10388000002AF7D1034800688862024801600020DE
:10389000ECE700003000002010B50548046803E0A4
:1038A0002046FFF76BFEA46A002CF9D110BD000082
:1038B0003000002001490860704700000C00002023
:1038C00010B504464FF47A7104FB01F000F002F8E1
:1038D00010BD000070B5034600224FF0E026756968
:1038E0000D4E366803FB06F44FF0E026B16910E098
:1038F0004FF0E026B06988420BD0884202D20E1AFF
:10390000324402E02E1A0E4432440146A24200D351
:1039100000E0EDE700BF70BD0C00002038B50446A4
:103920000D4600BF00BF1248C06940F001001049B9
:10393000C8610846C06900F00100009000BF00BFE8
:1039400000BF88040B49086008464560002181607B
:10395000C460FEF751F9002202211C20FDF767FD2B
:103960001C20FDF754FD0348FEF77AF938BD00002E
:103970000010024094010020FDF70EFD4FF4E0100E
:1039800000F048F84820FFF795FFFEF72FFFFEF7FD
:103990005FFDFFF727FDFFF74DF8FFF701F8FFF791
:1039A00029F841F61F413120FFF7B8FF1348FEF711
:1039B000C7FD21E012480078012802D100201049FB
:1039C00008701048007830B10E4800780E49087031
:1039D00000200C4908700C480078FFF7F3F800202D
:1039E00009490870094800680949884204D9FDF767
:1039F00071FD002005490860DCE700002D25000866
:103A00000600002004000020050000200000002027
:103A100040420F0030B58FB005460124282105A88B
:103A2000FCF77FFC14216846FCF77BFC0120059025
:103A3000000406900020079002200C90C1030D9115
:103A40000E9505A8FDF78CFE04460CB100BFFEE7FD
:103A50000F20009002200190002002904FF480601F
:103A600003900020049002216846FDF755FD0446AE
:103A70000CB100BFFEE70FB030BD00000000000039
:103A8000000001020304060708090000000001020B
:103A9000030402030405060708090A0B0C0D0E0FA8
:103AA000101001020010014000010001030000009D
:103AB00001000000001001400002000103000000AE
:103AC00001000000000801400002000103000000A6
:103AD0000100000000080140000800010300000090
:103AE0000100000000080140008000010300000008
:103AF0000100000000100140000800010300000068
:103B0000010000000014014001000001030000005A
:103B10000100000000140140040000010300000047
:103B2000010000000014014010000001030000002B
:103B300001000000001401404000000103000000EB
:103B4000010000000010014080000001030000009F
:103B50000100000000080140000100010300000016
:103B60000100000000080140000400010300000003
:103B700001000000000801400010000103000000E7
:103B800001000000001001400004000103000000DB
:103B900001000000001001400010000103000000BF
:103BA00001000000001401400200000103000000B9
:103BB00001000000001401400800000103000000A3
:103BC000010000000014014020000001030000007B
:103BD000010000000014014080000001030000000B
:103BE000010000000010000000140140010000006E
:103BF0000008000000140140020000000004000062
:103C000000140140030000000020000000140140E7
:103C1000070000000001000000140140080000003F
:103C200000800000000C01400400000008000000BB
:103C3000000C01400900000000C1814001C080412A
:103C400001C0804100C1814001C0804100C181406C
:103C500000C1814001C0804101C0804100C181405C
:103C600000C1814001C0804100C1814001C080414C
:103C700001C0804100C1814001C0804100C181403C
:103C800000C1814001C0804100C1814001C080412C
:103C900001C0804100C1814000C1814001C080411C
:103CA00001C0804100C1814001C0804100C181400C
:103CB00000C1814001C0804101C0804100C18140FC
:103CC00000C1814001C0804100C1814001C08041EC
:103CD00001C0804100C1814000C1814001C08041DC
:103CE00001C0804100C1814001C0804100C18140CC
:103CF00000C1814001C0804100C1814001C08041BC
:103D000001C0804100C1814001C0804100C18140AB
:103D100000C1814001C0804101C0804100C181409B
:103D200000C1814001C0804100C1814001C080418B
:103D300001C0804100C1814000C0C101C30302C273
:103D4000C60607C705C5C404CC0C0DCD0FCFCE0EDB
:103D50000ACACB0BC90908C8D81819D91BDBDA1A4B
:103D60001EDEDF1FDD1D1CDC14D4D515D71716D6BB
:103D7000D21213D311D1D010F03031F133F3F2322B
:103D800036F6F737F53534F43CFCFD3DFF3F3EFE9B
:103D9000FA3A3BFB39F9F83828E8E929EB2B2AEA0B
:103DA000EE2E2FEF2DEDEC2CE42425E527E7E6267B
:103DB00022E2E323E12120E0A06061A163A3A262EB
:103DC00066A6A767A56564A46CACAD6DAF6F6EAE5B
:103DD000AA6A6BAB69A9A86878B8B979BB7B7ABACB
:103DE000BE7E7FBF7DBDBC7CB47475B577B7B6763B
:103DF00072B2B373B17170B05090915193535292AB
:103E000096565797559594549C5C5D9D5F9F9E5E1A
:103E10005A9A9B5B99595898884849894B8B8A4A8A
:103E20004E8E8F4F8D4D4C8C4484854587474686FA
:103E30008242438341818040583E000800000020B8
:103E4000500000006C010008A83E0008500000204F
:103E5000303300008801000800000000000000006E
:103E60000024F4000000000000000000000000003A
:103E70000000000010000000010000000000000031
:103E80000000000000000000000000000000000032
:103E90000000000000000000000000000000000022
:083EA00000000000000000001A
:0400000508000131BD
:00000001FF
